:100000000C94E5020C941D030C941D030C941D0329
:100010000C941D030C941D030C941D030C941D03E0
:100020000C941D030C941D030C94B5270C94872885
:100030000C9494220C941D030C941D030C941D032A
:100040000C941D030C941D030C941D030C941D03B0
:100050000C941D030C941C230C941D030C941D0381
:100060000C941D030C941D030C941D030C941D0390
:100070000C941D030C941D030C941D030C941D0380
:100080000C941D030C941D030C941D030C941D0370
:100090000C941D030C941D030C941D030C941D0360
:1000A0000C941D030C941D030C941D036D056D052C
:1000B0009905990501061F06370737072A06C30663
:1000C000D406D406F4281B29132A1B29132A6729CE
:1000D0008A29132AE129F02929003A003B003C0033
:1000E0003D003E003F00400041004200430044000C
:1000F000450046004700480035001E001F00200054
:1001000021002200230024002500260027002D00C6
:100110002E002A0049004A004B002B0014001A0050
:100120000800150017001C0018000C001200130036
:100130002F00300031004C004D004E00390004000B
:100140001600070009000A000B000D000E000F004A
:100150003300340032002800E10064001D001B0061
:1001600006001900050011001000360037003800A5
:10017000E5005200E000E300E2002C00E600E700AA
:100180006500E400500051004F0000000100010034
:100190000100010001000100010001000100010057
:1001A0000100010001000100010001000100010047
:1001B0000100010001000100010001000100010037
:1001C0000100010001000100010001000100010027
:1001D0000100010001000100010001000100010017
:1001E0000100010001000100010001000100010007
:1001F00001000100010001000100010001000100F7
:1002000001000100010001000100010001000100E6
:1002100001000100010001000100010001000100D6
:1002200001000100010001000100010001000100C6
:1002300001000100010001000100010001000000B7
:1002400000047F3F1F643214643214783C1E1E1475
:100250000A052223252628292A2C2D2F3032333532
:1002600036383A3B3D3E4042434547494A4C4E5062
:1002700051535557595A5C5E6062646668696B6D8C
:100280006F71737577797B7D7F81838587898A8C90
:100290008E90929496989A9C9E9FA1A3A5A7A8AA97
:1002A000ACAEAFB1B3B4B6B8B9BBBCBEBFC1C2C3CC
:1002B000C5C6C7C9CACBCCCDCED0D1D2D2D3D4D566
:1002C000D6D7D7D8D9D9DADADBDBDBDCDCDCDCDC8F
:1002D000DDDDDDDDDCDCDCDCDCDBDBDBDADAD9D967
:1002E000D8D7D7D6D5D4D3D2D2D1D0CECDCCCBCAF5
:1002F000C9C7C6C5C3C2C1BFBEBCBBB9B8B6B4B31B
:10030000B1AFAEACAAA8A7A5A3A19F9E9C9A9896B0
:100310009492908E8C8A89878583817F7D7B797783
:100320007573716F6D6B6968666462605E5C5A5963
:1003300057555351504E4C4A4947454342403E3D24
:100340003B3A3836353332302F2D2C2A29282625B2
:100350002322FFAA7F554000010101010101010193
:100360000102020202020202020203030303030368
:100370000303040404040404040505050505060636
:1003800006060607070707070808080809090909F4
:100390000A0A0A0B0B0B0C0C0C0D0D0D0E0E0E0F9A
:1003A0000F0F10101111111212131314141515162A
:1003B000161717181819191A1A1B1B1C1D1D1E1E9B
:1003C0001F202021222223242425262627282929EC
:1003D0002A2B2C2D2D2E2F30313232333435363717
:1003E00038393A3B3C3D3E3F404142434445464715
:1003F00048494A4C4D4E4F50515354555658595AEE
:100400005B5D5E5F616264656668696B6C6D6F7091
:1004100072737577787A7B7D7E8082838587888A00
:100420008C8E8F91939596989A9C9EA0A2A3A5A737
:10043000A9ABADAFB1B3B5B7BABCBEC0C2C4C6C933
:10044000CBCDCFD1D4D6D8DBDDDFE2E4E7E9EBEEEC
:10045000F0F3F5F8FAFDFF0A0343004200380037D5
:100460000000001E034300680065007200720079FE
:100470000042002000530074007500640069006FA2
:100480000000000403090409023B00020100A0FA75
:1004900009040000010301010009211101000122EA
:1004A0004000070581030800010904010001030061
:1004B000000009211101000122B600070582032076
:1004C000000112010002000000084243878701007A
:1004D0000102000105010902A10185020901A10033
:1004E00005091901290815002501950875018102E2
:1004F0000501093009311581257F950275088106AE
:1005000009381581257F950175088106050C0A3883
:10051000021581257F950175088106C0C005010976
:1005200080A101850319012AB700150126B700959E
:100530000175108100C0050C0901A1018504190194
:100540002AA002150126A002950175108100C005A0
:10055000010906A1018506050719E029E71500250F
:10056000019508750181020507190029EF1500257D
:100570000195F07501810205081901290595057598
:10058000019102950175039101C005010906A101C0
:10059000050719E029E71500250195087501810275
:1005A0009501750881010507190029FF150026FF2F
:1005B000009506750881000508190129059505753E
:1005C000019102950175039101C011241FBECFEF67
:1005D000DAE0DEBFCDBF04B603FE18C08091710320
:1005E00090917203A0917303B09174038730904B84
:1005F000A740B04B59F410927103109272031092FD
:10060000730310927403E0E0F8E3099511E0A0E0B1
:10061000B1E0ECEAF6E502C005900D92A63CB10708
:10062000D9F723E0A6ECB1E001C01D92A137B207D3
:10063000E1F70E9449130C94542B0C94000081E0C4
:10064000089581E008950C94210308950C942503E6
:100650001F93CF93DF9300D000D01F92CDB7DEB7AA
:1006600049835A836B833091C90189819A81311101
:1006700014C0662359F0222349F00E947409182FF0
:10068000682F89819A810E941D0903C00E94480930
:10069000182F69817A81812F04C00E9474096981B1
:1006A0007A810F900F900F900F900F90DF91CF9164
:1006B0001F910C94B410FC01262F4081518162815E
:1006C000738184810C94280381E00895CF93DF9394
:1006D000EC0160E00E945B03BE01DF91CF910C94BE
:1006E00026030C94FA110C94F61108950E94C70782
:1006F0000E9475032FEF84E39CE0215080409040DE
:10070000E1F700C000000C9442230F931F93CF9396
:10071000DF938C0161E00E945B03EC01B8010E9451
:100720002303882309F44BC0B801CE010E94CD1DDC
:10073000882309F444C0B801CE010E94DF20882339
:10074000F1F1B801CE010E94F31E8823C1F1B80176
:10075000CE010E943B20882391F1B801CE010E9476
:10076000111C882361F1F8018281882309F1CB35BE
:100770008DE5D807C1F050F4C115FCE5DF0781F025
:10078000CF3DDC45A9F40E94AB0E19C0CC35EDE598
:10079000DE0761F0CD35DD4559F40E94EE0D08C04D
:1007A0000E9476030CC00E94F70D02C00E94FA0D51
:1007B000C801DF91CF911F910F910C941F0380E02E
:1007C000DF91CF911F910F9108950E94762280E0D2
:1007D0000E94021E0C9418040E94F11C0E941B042B
:1007E0000C947C2208950C94F20381E00895CF9339
:1007F000C82F0E94F503882359F0C095C1FF02C09D
:10080000889A01C08898C2FF02C08C9A01C08C9857
:10081000CF910895809A889A849A8C9A0895CF935C
:10082000C82F0E94F3038C2F0E94F703CF910895E5
:1008300080E00C940F040E943B210C940F040E9452
:100840003B219091C801891721F08093C8010C9435
:100850000F040895CF93DF93CDB7DEB72B970FB674
:10086000F894DEBF0FBECDBF4F83588769877A8764
:100870008B8761110E943A0D9E012F5F3F4F86E0EA
:10088000F90111928A95E9F785E0FE013796D901C1
:1008900001900D928A95E1F789819A814C815D8161
:1008A000452B31F09F3F31F491E08F3F19F403C0A5
:1008B00091E001C090E090FF09C049815A816B81AD
:1008C0007C818D819E810E945B0C05C0C9010E94C4
:1008D00064038111F2CF2B960FB6F894DEBF0FBEE2
:1008E000CDBFDF91CF910895FC01808191810E945D
:1008F000B6090895CF93882309F450C0C82F8CEF10
:100900008C0F813AD0F46C2F8091020190910301F9
:100910000E94B121882349F06C2F809102019091AF
:1009200003010E943C220E945C0D6C2F8091020109
:10093000909103010E9431220CC080E28C0F88301C
:1009400058F4C77081E001C0880FCA95EAF70E9489
:100950001D0DCF910C945C0DEBE5EC0FE33040F4F2
:10096000F0E0E65AFE4F808190E0CF910C946F2129
:10097000E8E5EC0FE73150F4F0E0EE0FFF1FE45D27
:10098000FE4F80819181CF910C948521CD3E30F036
:100990008C2F0E94CE13CF910C94A014CF91089568
:1009A000882389F19CEF980F913A40F4682F809149
:1009B0000201909103010E943C220DC090E2980F29
:1009C000983058F4877091E001C0990F8A95EAF742
:1009D000892F0E94230D0C945C0D9BE5980F93309A
:1009E00020F480E090E00C946F2198E5980F973107
:1009F00020F480E090E00C9485218D3E20F00E9450
:100A000029140C94A01408951F93CF93DF93182FEB
:100A1000EB010E947A04209741F08FE99FE0019753
:100A2000F1F700C000002197F6CF812FDF91CF9121
:100A30001F910C94D004893319F060E070E002C07B
:100A400060E570E00C940405882321F00E941D0DE0
:100A50000C945C0D0895882321F00E94230D0C94C2
:100A60005C0D0895CF92DF92EF92FF920F931F9348
:100A7000CF93DF937C01D62FC72FFC011281058114
:100A800002950F700E94130D8823B9F01123A9F06D
:100A90008C2F807F803421F080E28D0F883068F0C9
:100AA0008091F30282FD09C082E00E94BC0D0E9489
:100AB000130D91E0D82ED92601C0D12CCC2EC29492
:100AC0008FE0C8228C2D90E08C30910508F0CFC1CA
:100AD000FC01EA5AFF4F0C94AF2A8C2F807FCF7015
:100AE000882311F0C295C07F112399F0CC2309F41B
:100AF000AAC180E28D0F883010F0D11104C08C2F74
:100B00000E941D0D03C08C2F0E942D0D0E945C0DB4
:100B10009AC18D2F0E94D004CC2309F4A8C180E291
:100B20008D0F883038F1DD2329F18C2F0E94330D91
:100B300024C08C2F807FCF70803211F0C295C07F8F
:100B4000DD2319F0D130A1F13DC08091F30282FF85
:100B500017C0112349F0CC2329F08C2F0E941D0DC2
:100B60000E945C0D80E070C180E00E94D004CC2324
:100B700009F47DC18C2F0E94230D0E945C0D77C16A
:100B8000112371F0002341F0013031F40E943D0D3A
:100B90008C2B0E94450D6BC10E943D0D8C2B1DC0FE
:100BA000002319F0013009F462C10E94520D25C0E2
:100BB000112321F0063008F05AC10EC0053008F0AC
:100BC00056C11BC0112361F0002331F0F70185816C
:100BD00080FF39C18F7085838C2F0E94240547C107
:100BE000002359F0D93309F03FC1FFEF07EE13E0BE
:100BF000F15000401040E1F735C18C2F0E942B05C9
:100C000036C18C2F86958695837019F0813061F0FE
:100C10002EC1112321F08D2F9C2F937002C080E0F4
:100C200090E00E946F212BC1112321F08D2F9C2F6A
:100C3000937002C080E090E00E94852120C18D2F3A
:100C4000112319F00E94CE1302C00E9429140E94A1
:100C5000A01415C18C2F837009F047C011110BC16E
:100C60002D2F229526952770220F220F6D2F6F7042
:100C7000862F90E0A0E0B0E0022E04C0880F991FFC
:100C8000AA1FBB1F0A94D2F7D4FF10C04FE050E058
:100C900060E070E004C0440F551F661F771F2A955F
:100CA000D2F7409550956095709503C040E050E0B4
:100CB000BA01C695C695C3708A019B01082B192BF2
:100CC0002A2B3B2BC901B801C23049F058F4C1307E
:100CD00019F00E943308CFC00E942108CCC00E94A6
:100CE0004508C9C00E941F08C6C0112319F08C2FE7
:100CF000817001C08695882309F4BDC02D2F2295EF
:100D000026952770220F220F6D2F6F70862F90E08F
:100D1000A0E0B0E0022E04C0880F991FAA1FBB1FDD
:100D20000A94D2F7D4FF10C04FE050E060E070E0CA
:100D300004C0440F551F661F771F2A95D2F74095B0
:100D400050956095709503C040E050E0BA01C6959B
:100D5000C695C3708A019B01082B192B2A2B3B2BAC
:100D6000C901B801C23049F058F4C13019F00E94ED
:100D7000F80881C00E94E6087EC00E940A097BC074
:100D80000E94590878C0CF70112339F08C2F0E942F
:100D90007F088D2F0E9424056EC08D2F0E942B0589
:100DA0008C2F0E94A00867C0D23F21F128F4D03FC9
:100DB00041F0D13FC1F043C0D33F19F1D43F79F0A6
:100DC0003EC0112341F0053008F051C08C2F8F71C7
:100DD0000E94C5084CC0063008F049C0F7CF80918A
:100DE000F30282FF18C0112339F08C2F8F710E94FB
:100DF0007F083DC01123C9F38C2F8F710E94A0087A
:100E000036C0112329F08C2F8F710E946A082FC0E1
:100E10000E9465082CC0112349F0CF718C2F0E94CD
:100E20007F0863E08C2F0E94A10D21C081E00E9409
:100E3000BC0D0230E0F082E00E94BC0D18C011230E
:100E400031F0002391F28D2F0E947A0410C000230C
:100E500099F2D93349F41FEF27EE33E011502040C7
:100E60003040E1F700C000008D2F0E94D00488EFD1
:100E70008C0D843020F40E943B210E940F04DD2061
:100E8000C9F00E940F0D80FD15C0F70112820E946B
:100E9000090D0E947F08C7010E947B070E94090D6F
:100EA000DF91CF911F910F91FF90EF90DF90CF9046
:100EB0000C94A008DF91CF911F910F91FF90EF90BC
:100EC000DF90CF9008950F931F93CF93DF93EC01A2
:100ED000688179818A810E94C1098C010E941C0964
:100EE0000E940D08B801CE010E943205DF91CF911A
:100EF0001F910F910895CF93DF93EC019881898121
:100F00002B813C81232B31F08F3F31F481E09F3FD7
:100F100019F403C081E001C080E080FD1DC0CE0156
:100F20000E948503811110C00E94130D8823A1F037
:100F30008A81882389F08091F30282FD0DC082E0CE
:100F4000DF91CF910C94BC0DCE010E946307CE01BE
:100F5000DF91CF910C946603DF91CF91089580E0EB
:100F600090E00E946F2180E090E00E9485210E9425
:100F70003A0D0E945C0D0E94D1150C94A014809132
:100F80000201909103010E9447220C94AF070E9436
:100F90002A0D0C94BF0792959F70963079F010F44B
:100FA000925001C09A50923068F4803F69F018F472
:100FB000883E40F409C0843F29F406C0883E20F0F2
:100FC000813F11F080E0089581E00895FC01808167
:100FD00091810E94B6090E94CB070895CF93DF93B9
:100FE00000D000D01F92CDB7DEB70F900F900F90BA
:100FF0000F900F90DF91CF910895CF93DF9300D0A2
:1010000000D000D0CDB7DEB726960FB6F894DEBF7D
:101010000FBECDBFDF91CF910895089508950C9430
:101020000E080C940F080E94110860930A02709336
:101030000B0280930C0290930D020C94AF070C945A
:1010400013080F931F9300910A0210910B02209135
:101050000C0230910D02602B712B822B932B1F9170
:101060000F910C9413080F931F9300910A02109193
:101070000B0220910C0230910D0260237123822318
:1010800093231F910F910C9413080F931F930091BA
:101090000A0210910B0220910C0230910D02602780
:1010A0007127822793271F910F910C9413080C949A
:1010B0000E080E94570860930602709307028093FF
:1010C0000802909309020C94AF0760E070E0CB0136
:1010D0000C9459080F931F9341E050E060E070E0DA
:1010E0008A019B0104C0000F111F221F331F8A9524
:1010F000D2F7C901B8011F910F910C9459080F93B1
:101100001F9341E050E060E070E004C0440F551FC1
:10111000661F771F8A95D2F7809106029091070289
:10112000A0910802B09109028A019B01082B192B9A
:101130002A2B3B2BC901B8011F910F910C94590820
:101140000F931F9341E050E060E070E004C0440F53
:10115000551F661F771F8A95D2F740955095609569
:1011600070958091060290910702A0910802B091BB
:1011700009028A019B01082319232A233B23C90161
:10118000B8011F910F910C9459080F931F9341E0E0
:1011900050E060E070E004C0440F551F661F771FE9
:1011A0008A95D2F78091060290910702A0910802D9
:1011B000B09109028A019B01082719272A273B279A
:1011C000C901B8011F910F910C9459080F931F93F7
:1011D0000091060210910702209108023091090245
:1011E000602B712B822B932B1F910F910C9459081C
:1011F0000F931F930091060210910702209108029D
:101200003091090260237123822393231F910F9150
:101210000C9459080F931F93009106021091070236
:1012200020910802309109026027712782279327B5
:101230001F910F910C94590808952AE0929F800DF8
:101240001124E82FE695E695E695877051E001C0F8
:10125000550F8A95EAF785E0E89FF0011124E653DF
:10126000FE4F20E030E070E04081CB01022E02C052
:10127000969587950A94E2F7817081958427852356
:10128000842781932F5F3F4F2530310569F70895FB
:101290002AE0929F800D1124682F669566956695C9
:1012A000982F977085E0689FB001112440E050E0CE
:1012B00080E0FB01E40FF51FE653FE4F208130E094
:1012C000092E02C0369527950A94E2F7217033273C
:1012D000042E01C0220F0A94EAF7822B4F5F5F4F62
:1012E0004530510531F70895BF92CF92DF92EF92CA
:1012F000FF920F931F93CF93DF938C01C090060250
:10130000D0900702E0900802F090090280910A0252
:1013100090910B02A0910C02B0910D02C82AD92A1B
:10132000EA2AFB2ACFE1D0E0D701C6010C2E04C087
:10133000B695A795979587950A94D2F780FD04C036
:10134000219790F7B12C07C0BC2EB8018C2F0E94BA
:10135000C7100197A9F38B2DDF91CF911F910F91AA
:10136000FF90EF90DF90CF90BF900895CF93DF93E1
:10137000EC010E947409BE010E94C710DF91CF9159
:1013800008951F93CF93DF93EB019091C9019923A7
:1013900021F0CB010E94B60913C0882349F0CB018C
:1013A0000E947409182F682FCE010E941D0904C0E5
:1013B000CB010E944809182FBE01812F0E94C7103F
:1013C000DF91CF911F9108951F93CF93DF93C09129
:1013D0000E0216E080910F02C81799F0D0E01C9F12
:1013E000F0011D9FF00D1124E05FFD4F4081518100
:1013F00062817381848195810E94FD072196C77067
:10140000E9CFDF91CF911F91089540914002509113
:101410004102609142027091430280914402909196
:1014200045020C94FD07EF92FF920F931F93CF9309
:10143000DF938091450282958F7009F065C080919D
:101440004202882309F460C080910E02F0900F02DE
:101450001091400200914102609143027091440258
:1014600091E01F3F09F090E0C0910001D09101018F
:10147000292F96E0E92E8F1509F446C061157105F4
:1014800021F00F3F21F030E003C031E001C0322FE6
:1014900090E030FD36C0E89EF001E99EF00D112489
:1014A000DF01A05FBD4F11963C911197301329C009
:1014B0003C91311326C012963C911297311121C0F4
:1014C00013964D915C911497461B570B4C175D0773
:1014D000C0F4809145028F70806180934502EB5E7D
:1014E000FD4F80818F708061808380E492E00E9454
:1014F0007B07DF91CF911F910F91FF90EF900C949C
:10150000E40901968770B7CFDF91CF911F910F91BA
:10151000FF90EF9008959F92AF92BF92CF92DF928B
:10152000EF92FF920F931F93CF93DF93CDB7DEB768
:1015300061970FB6F894DEBF0FBECDBF8C0185E07A
:10154000F801DE011D9601900D928A95E1F7D80110
:101550001296EC9090914002E0914102209143025A
:10156000309144022115310531F0EF3F31F481E033
:101570009F3F19F403C081E001C080E0B82FB17033
:101580009B2E80FD47C1D8014C9111965C9111971B
:101590001396AD90BC90149780E4C82E82E0D82EAC
:1015A000F0904202B501621B730B20910001309153
:1015B0000101FF2009F4D9C0809145026217730729
:1015C00008F095C0282F207F09F052C05E1313C089
:1015D000491311C0FE2CE1100EC08F708061809302
:1015E00045020E94050AC6010E947B0780914502C0
:1015F000F80185834DC1AB2831F05F3F31F481E0C4
:101600004F3F19F403C081E001C080E080FD03C0BA
:1016100081E08E2502C080E090E0F82FF170FF2E6F
:1016200080FF1CC080910E0220910F0236E08217CD
:1016300009F40BC190E0389FF001399FF00D11249F
:10164000E05FFD4F6181561306C06081461303C001
:101650006281E61203C001968770E9CFFE2CEE206E
:1016600009F416C18091450281608093450254C0FF
:101670005E1306C0491304C0E11002C0F80199C00E
:10168000C8010E94E607882361F1EE2051F1209104
:101690004502822F82958F7090E0029774F08091BE
:1016A00040029091410298878F831986BB86AA8653
:1016B0002C87CE0107960E947B0786E0F801A0E404
:1016C000B2E001900D928A95E1F70E94130A0E9400
:1016D000050A0AC05E1711F1C8010E94E6078111D0
:1016E0002CC0C8010E947B07FF24F394D1C0282F8F
:1016F000207F81F77A2DB98AA88A6E2D89890E9468
:10170000EE0780E492E00E947B0786E0D6011D92FE
:101710008A95E9F70E94050AF12CBAC04913DCCF7B
:10172000E110DACFF8018583C8010E947B0786E0CB
:10173000D6011D928A95E9F7ABC0EE2091F2209177
:101740004502822F82958F7090E002970CF4B5CFFE
:1017500080914002909141029A8389831B82BD82CD
:10176000AC822E83CE010196A6CF6217730708F0D4
:1017700044C0FE2CEE2009F4B4CF5E1330C04913F0
:101780002EC02091450220FD21C0822F82958F70AE
:10179000482F50E041155105C9F0F80125834F301D
:1017A000510541F08F5F982F9295907F822F8F7017
:1017B000892B8583C8010E947B0786E0F801A0E49D
:1017C000B2E001900D928A95E1F73CC086E0F80105
:1017D000A0E4B2E001900D928A95E1F759C0C801EA
:1017E0000E94E607811169CF809145028160809354
:1017F0004502C8010E947B074BC07A2DB98AA88A8E
:101800006E2D89890E94EE0786E0D6011D928A9589
:10181000E9F718C0EE2009F464CFC8010E94E6077A
:10182000F82E882309F45DCF86E0F801A0E4B2E049
:1018300001900D928A95E1F780E492E00E94740491
:101840000E94130A0E94050A23C04D875E878D857A
:101850009E850E94B609292F22952F70223028F4E8
:101860009F7039F0811105C00BC0243028F49F709F
:1018700049F4805E883020F0C8010E947B079F2CCD
:10188000F92C06C0D80115969C91907F91F7F8CF5E
:101890008F2D61960FB6F894DEBF0FBECDBFDF91DE
:1018A000CF911F910F91FF90EF90DF90CF90BF905D
:1018B000AF909F9008951F93CF93DF93CDB7DEB77E
:1018C0002C970FB6F894DEBF0FBECDBF4F8358875D
:1018D00069877A878B879C87CE0107960E948B0A3F
:1018E0008823D1F09F8188852A853B85232B31F081
:1018F0008F3F31F481E09F3F19F403C081E001C0C4
:1019000080E080FD47C04F81588569857A858B8549
:101910009C850E94FD073EC086E0FE013796DE01F1
:10192000119601900D928A95E1F7FF81E8856A850D
:101930007B856115710531F0EF3F31F481E0FF3FA8
:1019400019F403C081E001C080E080FD23C0209134
:101950000F0230E0C90101968770992740910E026D
:1019600050E084179507F1F1F983EA837D836C8356
:1019700096E0929FD001939FB00D1124A05FBD4FC0
:10198000FE01319601900D929A95E1F780930F0236
:101990000E94E40916E080910E0290910F028917CF
:1019A00071F1189FC0011124805F9D4F0E948B0A26
:1019B000882329F1E0910E021E9FF0011124E05FBF
:1019C000FD4F4081518162817381848195810E94A4
:1019D000FD0780910E0290E0019687709927809311
:1019E0000E02D9CF0E94C70710920F0210920E026A
:1019F000E0E4F2E086E0DF011D928A95E9F72C969B
:101A00000FB6F894DEBF0FBECDBFDF91CF911F910F
:101A100008958091660285958595859508958091B4
:101A200066028770089590916602977081E009F4CC
:101A300080E0089580918902089590918902892B10
:101A400080938902089580959091890289238093DB
:101A50008902089510928902089590918802892B35
:101A600080938802089580959091880289238093BD
:101A7000880208951092880208958091670208955F
:101A800008950C94400D0C94410D9091F30292FD39
:101A900008C090916702981721F0809367020C9418
:101AA000430D089580916702882329F01092670200
:101AB00080E00C94430D0895CF93DF93E0910201F1
:101AC000F0910301809189028083E0910201F091FD
:101AD0000301908180918802892B80838091670225
:101AE000882381F0E0910201F09103019081892B1C
:101AF000808380910201909103010E949B218111BA
:101B00000E94520DC0910201D091030140E250E0C9
:101B100066E472E0CE010E94FF2A892B69F080E220
:101B2000FE01A6E4B2E001900D928A95E1F7CE01A4
:101B3000DF91CF910C944721DF91CF9108950C94C0
:101B4000400D9091F30292FD10C098E0899F9001A2
:101B50001124262B209366020E947F088091660242
:101B60008595859585950C949F0D0C947F08109212
:101B7000660280E00C949F0D20916602809582237E
:101B800080936602982F977099F430E0482F082EC2
:101B9000000C550B2417350759F09091F30292FD74
:101BA00007C08595859585950E94A0080C94B70D72
:101BB00008959091F30292FB222720F9281769F0EB
:101BC00080FB92F99093F3028091F2029091F302DC
:101BD0000E94270E82E00C94BC0D08958091F302C0
:101BE00082FB882780F991E089270C94D90D81E048
:101BF0000C94D90D80E00C94D90D6FEF7FEF80E04D
:101C000090E00C943E2B80E090E00E941A2B21E0A3
:101C1000893E9E4F09F020E0822F089582E090E0F7
:101C20000C940C2B83E090E00C940C2BCF9384E06D
:101C300090E00E940C2BC82F82E290E00E940C2BB7
:101C40002C2F30E0A901582BCA01CF910895CF93D2
:101C5000C92F682F84E090E00E94202B6C2F82E235
:101C600090E0CF910C94202BAB01BC018FE090E071
:101C70000C94322BAB01BC0183E190E00C94322B2D
:101C800060E070E0CB010C943A0E60E070E0CB01B4
:101C90000E94340E0C94400E69EE7EEF80E090E0DE
:101CA0000E943E2B60E082E090E00E94202B60E0EA
:101CB00083E090E00E94202B10920A0210920B0207
:101CC00010920C0210920D0260E084E090E00E94FD
:101CD000202B60E082E290E00E94202B60E085E013
:101CE00090E00E94202B60E086E090E00E94202B94
:101CF0006FEF87E090E00E94202B40E050E0BA01B7
:101D000088E090E00E94322B60E08DE090E00E943D
:101D1000202B40E050E0BA0188E190E00E94322B95
:101D200060E087E190E00E94202B40E050E0BA01A3
:101D30008CE190E00E94322B60E070E080E290E065
:101D40000E943E2B40E050E0BA0188E190E00E9402
:101D5000322B0C94450E0C944C0E682F8EE090E0C4
:101D60000C94202B0E9401236093A0027093A10287
:101D70008093A2029093A30260939C0270939D02B1
:101D800080939E0290939F02089585B7806885BFD7
:101D900085B7806885BF089581E008950C94CC0EC6
:101DA00008950C94D00E0C94D00E0C94D30E0C9479
:101DB000D00E0C94D70E0C94D00E0E94C50E83EA60
:101DC00091E10E9431210E94DB0E0C94D90E0E94F9
:101DD000D10E0C94D00E0E94BD110E940A040C94E6
:101DE000B81E0E94EC220E94A2120E94EB0E0E94DA
:101DF000F11C0E94301B0C94D50E5F926F927F9263
:101E00008F929F92AF92BF92CF92DF92EF92FF920A
:101E10000F931F93CF93DF93CDB7DEB72A970FB6FB
:101E2000F894DEBF0FBECDBF0E94B712C82E81113D
:101E30000E94B20E3AE8832E32E0932E00E010E0CA
:101E4000502E802F0E94E1115C01F401619071908D
:101E50004F016826792661147104B1F40F5F1F4F9A
:101E60000930110569F78FEF89838A831B820E94ED
:101E7000F5228160782F9D838C8349815A816B8103
:101E80008D810E942A043AC08091A40281FD0E94A3
:101E9000EA11D12CEE24E394F12CC3018E219F2171
:101EA000892B29F10E94CE0E8823A9F0DE825F8261
:101EB000AE20BF2081E0AB2809F480E088870E9433
:101EC000F5228160782F9A8789874E815F816885A6
:101ED0008A850E942A04000F111FF801E657FD4F62
:101EE00080819181E826F926F182E08207C0D394AF
:101EF000EE0CFF1CFAE0DF12D0CFB0CF81E0C110B2
:101F000001C080E02A960FB6F894DEBF0FBECDBFA9
:101F1000DF91CF911F910F91FF90EF90DF90CF90C5
:101F2000BF90AF909F908F907F906F905F9008953B
:101F30000E94FD0E0E94631B0E94B71E0E94BE14E9
:101F40000C941F04CF93DF930E94CC10EC018115F9
:101F500021E5920708F045C0811530E5930708F0A8
:101F600094C0883E910528F5803E910508F0F8C0A0
:101F7000883A910570F4853A910508F07CC081306B
:101F8000910509F475C008F4E8C0049708F0E8C0AA
:101F9000E4C08F3B910508F0E0C0C85AD0E0CC0FF8
:101FA000DD1FC35ADE4F0990D881C02DCE01946445
:101FB000D8C0811540E2940758F4811551E0950787
:101FC00008F0CEC08D3E910508F4C7C09065C9C029
:101FD000C11580E4D80708F4C0C0DF70CE01906A54
:101FE000C0C0811525E59207A8F4811534E5930753
:101FF00008F095C0811543E5940708F07BC0811572
:1020000052E5950708F061C0D82FCC27CE01816F2B
:10201000906AA7C0C11589E5D807A0F4C11528E5C5
:10202000D20708F082C0C11536E5D30708F095C085
:102030008C2F0E9460118F7190E0D82FCC27CE0199
:1020400090628FC0C1154AE5D40708F474C0CE0170
:1020500090568115904208F080C08D2F8F710E949C
:102060006011DD27D0628F71AE01582BCA0179C093
:1020700081E090E076C0C55AD0E0C557DE4F888138
:10208000C82FD0E0CE0190646CC074E0969587951F
:102090007A95E1F7282F23703C2F337081E090E090
:1020A00002C0880F991F3A95E2F79C68AC01522B49
:1020B0009A019C2F9F709695969550E2959FE0010E
:1020C0001124C9018C2B9D2B4CC08370992721E0D2
:1020D00030E002C0220F331F8A95E2F79C2F9695BD
:1020E000969580E2989FE0011124C22BD32BCE015C
:1020F0009C6837C08370992721E030E002C0220F2E
:10210000331F8A95E2F79C2F9695969540E2949F0F
:10211000E0011124C22BD32BCE019A6822C0D82F04
:10212000CC27CE01846F906A1CC0DC2FCC27CE0157
:10213000806F906A16C08C2F8F700E94601194E09F
:10214000D695C7959A95E1F7CF70D0E0DC2FCC27D4
:10215000D0699E01282BC90104C080E090E001C035
:10216000CE01DF91CF9108952AE5829FC00111240D
:10217000FC012AE0729FE00DF11D1124E60FF11D14
:10218000EE0FFF1FE852FF4F8591949108950E9432
:10219000B4100E94A20F08958238910569F1B0F43D
:1021A0008133910509F46DC048F48932910509F431
:1021B00063C08A32910509F469C008958533910599
:1021C00009F455C089339105B9F00895833E91050E
:1021D00069F138F4803E9105B1F0823E910509F134
:1021E0000895863E9105A9F1873E9105B9F1843E97
:1021F000910509F064C023C02091F20220FD4FC078
:1022000021FD4DC008958091F20280FD44C080916F
:10221000F30280FF44C08091F20284FD42C083EE4D
:102220004DC08091F20282FF38C0F5CF8091F2025A
:1022300082FD33C08091F30280FD31C0ECCF8091EC
:10224000F30281FF32C08091F20284FD2AC087EE42
:1022500035C08091F20283FF26C0F5CF8091F20253
:1022600083FD21C08091F30281FD1FC0ECCF8091DE
:10227000F20285FD1CC01DC08091F20285FD19C0CF
:1022800016C08091F20286FD16C017C08091F2023E
:1022900086FD13C010C089E311C082EE0FC080EE2E
:1022A0000DC080E00BC086EE09C084EE07C089E255
:1022B00005C085E303C08AE201C081E390E0089590
:1022C0009091F20292FF0DC0282F2871283019F446
:1022D000877F846006C0282F2471243011F48B7FFF
:1022E000886093FF0DC0282F2871283119F4877E4C
:1022F000846106C0282F2471243111F48B7E8861FB
:102300002091F30220FF0DC0382F3871383019F4B6
:10231000877F816006C0382F3171313011F48E7F94
:10232000886021FF0DC0282F2871283119F4877E7D
:10233000816106C0282F2171213111F48E7E8861C0
:1023400094FD877E089580E008950C94FD0D0E9411
:10235000B7128FE39CE90197F1F700C000000E94DB
:10236000B71280E00E94E11180FF04C00E94A51115
:102370000C94422308950C94A7110E94030E81111E
:1023800002C00E94AB0E0E940E0E8093A4020E9417
:10239000160E9093F3028093F2020E94BB110E94EA
:1023A000120E682F70E080E090E00E941F0860919C
:1023B00006027091070280910802909109020C9424
:1023C0005708E82FF0E0EE0FFF1FEA5FFC4F808117
:1023D00091810895089580EA8A95F1F7089500C0E3
:1023E00008950C94EB1108950C94F3110C94F411CE
:1023F0000C94F3110C94F811F894E82FE295EF7017
:10240000F0E031A1282F2F7081E090E001C0880F0B
:102410002A95EAF7982F9095932391A392A1892B5F
:1024200082A3789408950F931F93CF93DF93C8E905
:10243000D1E089918F3F11F00E94FC1181E0C13AF7
:10244000D807B9F7CEE8D1E008E911E089918F3FCC
:1024500011F00E94FC110C171D07C1F7DF91CF91FD
:102460001F910F910895BF92CF92DF92EF92FF924A
:102470000F931F93CF93DF938C01C62FD0E0CE0133
:1024800088569E4F6C01FC0190819F3F09F450C01B
:10249000B62EF894E92FE295EF70F0E081A19F70DD
:1024A00021E030E001C0220F9A95EAF7822B81A348
:1024B00082A12095282322A378940E94EF11EEE8B0
:1024C000F1E048E951E021E030E0E12CF12C6191AC
:1024D0006F3F89F0A62FA295AF70B0E090968C91D7
:1024E00090E06F7002C0959587956A95E2F780FD40
:1024F00002C0C90102C080E090E0E82AF92A220F58
:10250000331F4E175F0719F7F60180818F3F11F0D7
:102510000E94FC1161E0E114F10409F460E08B2DEC
:102520000E94F111CC0FDD1FC00FD11FF982E8828C
:10253000DF91CF911F910F91FF90EF90DF90CF909F
:10254000BF9008950E94131282E1E6E0F3E0DF01FC
:10255000982F1D929A95E9F7E4EFF2E0DF011D92C2
:102560008A95E9F789E00E9402130C947103FF92A7
:102570000F931F93CF93DF93CDB7DEB762970FB65C
:10258000F894DEBF0FBECDBF8E010F5F1F4F82E1FB
:10259000F80111928A95E9F7F12C6F2DC8010E947C
:1025A0003312F394F9E0FF12F8CF42E150E0B801A2
:1025B00084EF92E00E94FF2AFF24F394009709F42D
:1025C000F12C892B41F082E1F801A4EFB2E00190F7
:1025D0000D928A95E1F72F2D49E066E073E084EFD4
:1025E00092E00E9403130E9473038F2D62960FB630
:1025F000F894DEBF0FBECDBFDF91CF911F910F9139
:10260000FF9008950895FF920F931F93CF93DF9348
:10261000F82E092F162FD72FC42F222349F081E03F
:102620008093A7020E94F5229093A6028093A502B0
:102630008091A7028823D9F08091A5029091A602EB
:102640000E940D23059798F0EF2DF02FA12FBD2F9D
:1026500080E090E04C2F50E08417950734F42191EE
:1026600031912D933D930196F7CF1092A702DF9100
:10267000CF911F910F91FF9008950E940D250E9408
:10268000F10E0C9419250E941D250E94980F0C94A0
:1026900037250E9493220E94F4240E94DD0E0E949E
:1026A0003D130E9443130E94E70EFBCF8091AE02C0
:1026B00080FF06C06091090170E0660F771F26C099
:1026C00081FF04C06091090184E005C082FF07C05A
:1026D0006091090188E0689FB001112417C09091B2
:1026E000AD029923D1F060910801961788F72091E7
:1026F000090188E0289F90011124929FA001939FD7
:10270000500D112470E0CA010E94792A60387105C9
:1027100040F46115710519F406C068E070E0862F79
:1027200008958FE7089581E008958091AE0280FFBB
:1027300008C06091050170E075956795759567957E
:1027400021C081FF06C06091050170E07595679515
:1027500019C082FF04C06091050170E010C0909123
:10276000AC02992399F0609104019617A0F780912B
:102770000501899FC001112470E00E94792A603808
:10278000710540F46115710519F406C061E070E04F
:10279000862F08958FE7089581E008958D3E21F4F6
:1027A0000E945613819504C08E3E29F40E94561350
:1027B0008093B20208958F3E21F40E9456138195B2
:1027C00004C0803F29F40E9456138093B1020895FB
:1027D000893F19F40E94951305C08A3F31F40E9485
:1027E000951381958093B30208958B3F21F40E9445
:1027F0009513819504C08C3F29F40E949513809312
:10280000B40208959FE0980F983078F421E030E00A
:10281000A90102C0440F551F9A95E2F7CA01909191
:10282000B002892B8093B00208958D3F21F48091EE
:10283000AE0281600BC08E3F21F48091AE028260B7
:1028400005C08F3F29F48091AE0284608093AE0270
:1028500008958D3E39F49091B20297FF35C01092E1
:10286000B20259C08E3E29F49091B2021916BCF3FF
:102870002BC09091B1028F3E29F497FF25C0109292
:10288000B10249C0803F19F41916CCF31DC09091D4
:10289000B302893F29F41916BCF41092B3023BC06D
:1028A0008A3F19F497FF10C0F8CF8B3F39F490910D
:1028B000B40297FF09C01092B4022DC08C3F21F4DE
:1028C0009091B4021916BCF39FE0980F983080F4F1
:1028D00021E030E0A90102C0440F551F9A95E2F7AC
:1028E000CA0180959091B00289238093B00213C0F1
:1028F0008D3F21F48091AE028E7F0BC08E3F21F47C
:102900008091AE028D7F05C08F3F29F48091AE0289
:102910008B7F8093AE028091B102811106C08091BD
:10292000B202811102C01092AD028091B3028111F6
:1029300006C08091B402811102C01092AC020895C9
:102940000E94F5222091B102211104C02091B2020F
:10295000222321F09093AB028093AA022091B3022C
:10296000211104C02091B402222321F09093A902E6
:102970008093A8028FEA92E00C946121EF92FF927B
:102980000F931F93CF93DF9300D000D000D0CDB72B
:10299000DEB786E0EFEAF2E0DE01119601900D92DB
:1029A0008A95E1F7E090B102F090B2020091B30293
:1029B0001091B4021092B1021092B2021092B302BE
:1029C0001092B402E11003C0FF2009F45DC08091B1
:1029D000AA029091AB020E940D23AC019091AD022E
:1029E000992339F020910A0130E02417350758F077
:1029F0004BC020910B018AE0289F900111242417DD
:102A0000350718F041C09F3F19F09F5F9093AD02CA
:102A1000EE2061F00E9456131E1414F09FEF01C0C7
:102A200091E0989F902D11249093B102FF2061F0C6
:102A30000E9456131F1414F09FEF01C091E0989F5D
:102A4000902D11249093B2023091B1023323E1F022
:102A50002091B2022223C1F045EB3403C0011124BE
:102A6000992319F09093B10203C081E08093B102E1
:102A700035EB2303C0011124992319F09093B2027E
:102A800003C081E08093B202011103C0112309F455
:102A90005DC08091A8029091A9020E940D23AC0113
:102AA0009091AC02992339F02091060130E024176F
:102AB000350758F04BC0209107018AE0289F90010C
:102AC00011242417350718F041C09F3F19F09F5F6C
:102AD0009093AC02002361F00E949513101614F03D
:102AE0009FEF01C091E0989F902D11249093B30225
:102AF000112361F00E949513111614F09FEF01C08D
:102B000091E0989F902D11249093B4023091B302DC
:102B10003323E1F02091B4022223C1F045EB3403CA
:102B2000C0011124992319F09093B30203C081E0EE
:102B30008093B30235EB2303C0011124992319F0CC
:102B40009093B40203C081E08093B4028091B102FB
:102B500081110BC08091B202811107C08091B30234
:102B6000811103C08091B40281110E94A014EB82F4
:102B7000FC820D831E8386E0FE013196AFEAB2E04F
:102B800001900D928A95E1F726960FB6F894DEBF74
:102B90000FBECDBFDF91CF911F910F91FF90EF90AE
:102BA0000895EFEAF2E086E0DF011D928A95E9F7E9
:102BB0001092AD021092AC021092AE020895EF9204
:102BC000FF920F931F93CF93DF938B01682F111107
:102BD0000AC0442329F0E82FF0E0E95AFC4F649141
:102BE000762F862F75C0212F30E0E82FF0E04423A8
:102BF00021F0E95AFC4FE491F0E046E0049FC00167
:102C00001124CFEFD0E0BE010E94652A4BEA4603B3
:102C1000C001479F900D1124800F911D800F911DC1
:102C2000982F990F890FAE01421B530B4E9FD00175
:102C30004F9FB00D5E9FB00D11249B2F189FA001D8
:102C40001124452F55278E01041B150B0E9FA00143
:102C50000F9F500D1E9F500D11247E01E81AF108A0
:102C6000E29E8001E39E100DF29E100D1124212F93
:102C70003327C21BD30BCE9F9001CF9F300DDE9F19
:102C8000300D112462307105A9F048F46115710509
:102C900069F061307105C9F48B2F752F0DC0643058
:102CA000710581F058F06630710579F47E2F8B2F15
:102CB000932F0DC0832F7B2F9E2F09C08E2F7B2F2C
:102CC000952F05C08E2F732F02C07E2F852F692F61
:102CD000DF91CF911F910F91FF90EF90089541E008
:102CE0000E94DF15089508950E946F160895CF93EE
:102CF000DF93762FE901682F842F0E947416798361
:102D000068838A83DF91CF91089580911803282FDB
:102D1000269530E02115310519F48170826005C0D7
:102D20002532310524F0817088648093180308955A
:102D300088E090E00C94142BCF92DF92EF92FF92F8
:102D40006B017C010E948516B701A60188E090E026
:102D5000FF90EF90DF90CF900C94322BE8E1F3E0FE
:102D600083E0808311828FEF82838383148260816A
:102D70007181828193810C949C168091180380FF4D
:102D800002C08695089580E0089590911C039330C9
:102D900018F49F5F90931C03882351F060911803EF
:102DA0007091190380911A0390911B030C949C1647
:102DB000089581E00C94C51690911C03992319F095
:102DC000915090931C03882351F0609118037091E7
:102DD000190380911A0390911B030C949C1608957B
:102DE00081E00C94DC1670E00C94C81E6091100118
:102DF0008091180380FF0AC080910F0123E0829F19
:102E0000C0011124835E9C4F0C94F3168091110134
:102E100090911201891780F7E82FF0E09F01220FAF
:102E2000331FE20FF31FE35EFC4F11821082128208
:102E30008F5FF0CF9091180390FF16C09091110111
:102E400020911201921770F4E92FF0E0DF01AA0F30
:102E5000BB1FEA0FFB1FE35EFC4F8183608342834D
:102E60009F5FF0CF0C94F6160895CF93DF9300D0B8
:102E70001F92CDB7DEB79091180390FF0AC09E0154
:102E80002F5F3F4F0E9477164B8169818A810E9494
:102E90001A170F900F900F90DF91CF910895CF9355
:102EA000DF93EC01EC81F0E0EE5AFD4F4491E8E154
:102EB000F3E0628181810E9435178C818F5F8C8362
:102EC000DF91CF910895CF93DF93EC01E8E1F3E038
:102ED000438162818C810E9435178C818F5F8C8346
:102EE000DF91CF9108950F931F93CF93DF9300D07D
:102EF0001F92CDB7DEB78C018091B50281110AC057
:102F00009E012F5F3F4F4FEF6FEF0E9477168A8130
:102F10008093B502F8018481813051F028F082302D
:102F200061F44091B5020AC08091B50240E007C04B
:102F30006091B50240E080E003C040E080E060E0E6
:102F40000E941A17F801848190E0019663E070E016
:102F50000E94792A84830F900F900F90DF91CF9178
:102F60001F910F910895AF92BF92CF92DF92EF928F
:102F7000FF920F931F93CF93DF9300D01F92CDB793
:102F8000DEB7182FF62E042FE22E9091180390FF33
:102F90006DC0E92FE695AE2FB0E0AF55BE4F8C91D6
:102FA0008093BF029E7F923061F49E012F5F3F4F5E
:102FB000812F0E9477164B8169818A810E941A179E
:102FC00043C0823019F400911B033EC0863019F4CF
:102FD0001091190339C08930D9F38931A9F5E95124
:102FE0008E2F8170D82EE695F0E0EE5AFC4FA5901A
:102FF000B490C12CBB2460911301C61618F52C2D7A
:1030000030E0A29EC001A39E900DB29E900D1124AF
:1030100070E00E94652A812FD11002C0860F01C086
:10302000861B90911101290F311DA901440F551FD5
:10303000240F351F235E3C4F402F6F2D0E947716C3
:10304000C394D9CF0E94F61610931903F0921A0375
:1030500000931B03EE2051F0609118037091190347
:1030600080911A0390911B030E949C160F900F9061
:103070000F90DF91CF911F910F91FF90EF90DF9014
:10308000CF90BF90AF900895E8E1F3E09181282FB1
:103090004381628188E0890F0C94B31781E00C941E
:1030A0004418E8E1F3E09181282F4381628188EFA1
:1030B000890F0C94B31781E00C945118E8E1F3E008
:1030C000628128E0620F08F46FEF282F438181812D
:1030D0000C94B31781E00C945E18E8E1F3E0628190
:1030E00028E0621B08F460E0282F438181810C9462
:1030F000B31781E00C946D18E8E1F3E0438128E018
:10310000420F08F44FEF282F628181810C94B3178E
:1031100081E00C947C18E8E1F3E0438128E0421B55
:1031200008F440E0282F628181810C94B31781E07C
:103130000C948B1820E00C94B317FF920F931F93FD
:10314000CF93DF93EC01F12C0FEF10E060911301AE
:10315000F616F0F4809111012F2D30E0280F311D6B
:10316000C901880F991F280F391F235E3C4F70E05B
:10317000C8010E94792A962F8C8140911B0360918F
:103180001A03F99E800D11240E947716F394DECF66
:103190000E94F6169A818C8190FF02C08F5F01C059
:1031A00081508C83DF91CF911F910F91FF900895F3
:1031B000AF92BF92CF92DF92EF92FF920F931F9345
:1031C000CF93DF93FC01828180FF02C00FEF01C02B
:1031D00001E010E046E1A42E80911301181708F0D9
:1031E00043C080911101C12ED12CE601C80FD11D21
:1031F000CE01880F991FC80FD91FC35EDC4F1982FB
:1032000018821A8234E0E32EF12CB12C8091B7029F
:103210008B0D87312CF06A2D0E94572A892F05C00B
:1032200087FF03C090911301890F082E000C990BA2
:10323000C816D90691F480911B038E9DA0018F9D25
:10324000500D112455954795559547959E016091D0
:103250001A03809119030E947716B00EF1E0EF1A5D
:10326000F108A1F61F5FB8CF0E94F6168091B70251
:10327000013031F4811102C080911301815007C0E7
:1032800090E001966091130170E00E94792A80938A
:10329000B702DF91CF911F910F91FF90EF90DF90D8
:1032A000CF90BF90AF900895CF93809111019091EE
:1032B0001201891770F4E82FF0E09F01220F331FED
:1032C000E20FF31FE35EFC4F1182108212828F5FC8
:1032D000F0CFC0E060911301C617C0F5EC2FF0E00D
:1032E00070E0CF010E94792A20911101820F209174
:1032F000B602022E000C330B90E0E217F307CCF07D
:1033000020910E01022E000C330B2E173F078CF07C
:103310009C01220F331F820F931F9C01235E3C4FA1
:1033200040911B0360911A03809119030E94771644
:103330000BC0FC01EE0FFF1F8E0F9F1FFC01E35E11
:10334000FC4F118210821282CF5FC4CF0E94F6160A
:1033500020910D018091B602820F8093B602909168
:103360000E01920F90930E0119165CF4082E000CBA
:10337000990B4091130150E0415051098417950772
:103380001CF0219520930D01CF9108958F929F926B
:10339000AF92BF92CF92DF92EF92FF920F931F9363
:1033A000CF93DF938C01FC014481C42FD0E09E01B8
:1033B000DE010E94BD2A9B01AC010E94D32A6B0151
:1033C0007C01E0E2F0E0EC1BFD0BA5E5B0E09B0129
:1033D000AC010E94D32A4B015C019F01DF010E94D6
:1033E000B52A9B01AC010E94DE2A9B01AC012C0D89
:1033F0003D1D4E1D5F1DC501B4010E948D2AC22FC7
:10340000D22F2A3228F4F3E02F9F900111240DC00F
:1034100025E530E02C1B3109C901880F991F280FC1
:10342000391F37FF02C02F5F3F4F35952795C22FB9
:10343000C095F12C85E5E82EED1A80911301F81660
:10344000C8F4F1FC02C08E2D01C08D2F90911101A6
:103450002F2D30E0290F311DA901440F551F240FD6
:10346000351F235E3C4F4C2F60911A030E94771644
:10347000F394E3CF0E94F616F8018481811102C013
:1034800091E003C0803219F49FEF90930C0190916A
:103490000C01890FF8018483DF91CF911F910F9167
:1034A000FF90EF90DF90CF90BF90AF909F908F9064
:1034B00008950F931F93CF93DF93EC0100E010E08A
:1034C00080911301282F30E00217130724F5909103
:1034D00011019801290F311DA901440F551F240F17
:1034E000351F235E3C4F869590E04C8108171907E5
:1034F0001CF4442331F002C0411103C040911B036E
:1035000001C040E060911A03809119030E94771670
:103510000F5F1F4FD5CF0E94F6168C8190E0019669
:10352000817099278C83DF91CF911F910F9108951E
:10353000E8E1F3E080818E7F808360817181828108
:1035400093810E949C161092C0022FEF80E792E0B8
:10355000215080409040E1F700C000000C94F61626
:1035600060911803669570E04BE050E084E191E0D3
:103570000E94F22A892B19F481E08093C0020E94F4
:10358000F5229093B9028093B802089590911803A0
:1035900090FF35C09170811102C0926006C08532E3
:1035A00010F0986402C0880F982B9093180366233C
:1035B00051F0609118037091190380911A03909152
:1035C0001B030E949C1660911803669570E04BE007
:1035D00050E084E191E00E94F22A892B19F01092C8
:1035E000C00202C00E94B01A81E08093BB024091E9
:1035F0001B0360911A03809119030C949A18089583
:10360000682F90911803969581E0890F853208F014
:1036100081E00C94C61A81E00C94001B682F9091F5
:10362000180396958FEF890F09F484E20C94C61A5B
:1036300081E00C940E1B61E00C94C61AE8E1F3E003
:1036400080818160808386950C941B1B8091180378
:1036500080FD0C94981A0C941E1B60E00C94C61A02
:103660008091BE0281112EC00E94030E811104C000
:103670000E94AB0E0E94AE160E949816609318032B
:103680007093190380931A0390931B036E7F61F468
:103690000E94AE160E949816609318037093190347
:1036A00080931A0390931B030E9485161092C00208
:1036B0008091180380FF03C086950E942D1B81E036
:1036C0008093BE0208950F931F93CF93DF93809151
:1036D000C002882309F485C08091BF02E0911803DD
:1036E000E695E81BE093BA02823049F4F0E0E25B31
:1036F000FD4FE491CE2FD0E00FE417E149C08630B2
:1037000049F4F0E0E55BFD4FE491CE2FD0E003E615
:1037100017E13EC0893051F4E695F0E0E85BFD4FDB
:10372000E491CE2FD0E00DE918E132C08F3051F492
:10373000E695F0E0EB5BFD4FE491CE2FD0E008ED95
:1037400018E126C0853149F4F0E0EE5BFD4FE491CD
:10375000CE2FD0E004E519E11BC0883181F083321F
:1037600039F4E0E4F2E0C591D49103E717E110C029
:10377000843251F4C4EFD1E009E51AE109C0C8E28E
:10378000D0E006EC19E104C0C0EDD7E003E716E194
:103790008091BB02882361F01092BB020E94F52247
:1037A0009093B9028093B8021092BD021092BC02AD
:1037B0000E94F522E091B802F091B9028E1B9F0B96
:1037C0008F3F9F4770F4EC0FFD1FF093B902E09319
:1037D000B80288EB92E0F801DF91CF911F910F9131
:1037E0000994DF91CF911F910F910895882311F0D3
:1037F000FA0101C0FB010994CF93DF93C82FD62FA4
:103800000E94BD168C1740F00E94BD168D1720F443
:10381000DF91CF910C940B1B8C2FDF91CF910C94E7
:103820001B1B1F93CF93DF93FB0112811111C3C0A8
:10383000EC010E941A0D8272CD3CFCE5DF0709F411
:103840009AC0A8F5C73CECE5DE0709F476C0A8F4F9
:10385000C43C9CE5D90709F45FC028F4C33CDC45AF
:1038600009F457C054C0C53C9CE5D90709F459C0B8
:10387000C63CDC4509F45CC04AC0CA3CFCE5DF0735
:1038800009F46AC050F4C83CECE5DE0709F45AC0FC
:10389000C93CDC4509F45BC03AC0CB3C9CE5D90788
:1038A00009F45FC0CC3CDC4509F460C030C0C23DC7
:1038B000FCE5DF0709F46FC088F4CF3C9CE5D9072D
:1038C00009F460C008F45CC0C03DFCE5DF0709F402
:1038D0005CC0C13DDC4509F45BC019C0C53D9CE539
:1038E000D90709F460C050F4C33DFCE5DF0709F4D3
:1038F00055C0C43DDC4509F454C009C0C63D9CE533
:10390000D90709F455C0CE35DD4509F454C011E09E
:1039100052C00E94261B4FC048E15BE16BE07BE197
:1039200004C04BE05BE168E17BE10E94F61B43C011
:103930004BE558E16EE478E1F8CF4EE458E16BE5F1
:1039400078E1F3CF49E758E16AE678E1EECF4AE65D
:1039500058E169E778E1E9CF47E958E168E878E1BB
:10396000E4CF48E858E167E978E1DFCF40EF56E17E
:1039700069ED76E1DACF49ED56E160EF76E1D5CF3A
:1039800081E017C065E082E010C068E086E00DC00D
:103990006EE089E00AC064E18FE007C067E185E17D
:1039A00004C088E106C062E289E10E94FC1B03C0FA
:1039B00083E20E941B1B812FDF91CF911F910895FD
:1039C00086E090E00C940C2B682F86E090E00C943D
:1039D000202B80915F038470896180935F030C9436
:1039E000E41C0E94030E811104C00E94AB0E0E94D1
:1039F000E91C0E94E01C80935F03282F26952695E2
:103A0000269530E02430310524F08770886180935A
:103A10005F0380915F0380FF04C08695869586953D
:103A200001C080E00C94021E20915F03822F8695D6
:103A300086958695482F50E04330510554F48F5FAA
:103A4000982F990F990F990F822F8770892B809348
:103A50005F0380915F03816080935F030E94E41C99
:103A600080915F038695869586950C94021E8091C1
:103A70005F03982F969596959695A1F0915E990F74
:103A8000990F990F8770892B80935F03887F91E04E
:103A900009F490E080915F0390FB80F980935F03CD
:103AA0000E94E41C80915F038695869586950C9410
:103AB000021E80915F0380FD13C0816080935F03CD
:103AC000813019F489E080935F0380915F030E9445
:103AD000E41C80915F038695869586950C94021E62
:103AE000089580915F0380FF08C08E7F80935F03FD
:103AF0000E94E41C80E00C94021E089580915F03F4
:103B000080FD0C94711D0C94591D90915F03892FB9
:103B10008695869586958F5F8F719770843038F47F
:103B2000880F880F880F892B80935F0302C09093C2
:103B30005F0380915F03887F91E009F490E08091BA
:103B40005F0390FB80F980935F030E94E41C8091E7
:103B50005F038695869586950C94021E843008F046
:103B600083E090915F039770282F220F220F220F7E
:103B7000922B90935F03987F21E009F420E09091CD
:103B80005F0320FB90F990935F030C94021E0E9448
:103B9000AE1D80915F030C94E41C9C01FB018281AB
:103BA000882349F12E3BFCE53F07C9F040F42C3B4C
:103BB000ECE53E0769F02D3B3C4561F00895203C63
:103BC0009CE5390791F070F0213C3C4589F008955F
:103BD00083E001C080E00E94C71D80E008950E943C
:103BE000371DFBCF0E94141DF8CF0E947E1DF5CF1C
:103BF0000E94851DF2CF81E00895269A2E9808959F
:103C00002E9808958F929F92AF92BF92CF92DF929B
:103C1000EF92FF920F931F93CF93DF93C82F8430BF
:103C200050F4811109C0809180008F7D80938000C5
:103C30000E94001E06C0C3E08091800080628093D5
:103C40008000A0918600B09187002C2F30E00E9468
:103C5000BD2A23E030E040E050E00E948D2A00279A
:103C6000122F232F342F012F122F232F3327809130
:103C70008600909187006CE070E00E94652A6017D2
:103C8000710730F0C80169E070E00E94652A5EC0EB
:103C90008091860090918700E0908600F0908700E8
:103CA000E0918600F0918700C6E0D0E0BE010E945E
:103CB000652A060F171F211D311D4801590185E096
:103CC000880C991CAA1CBB1C8A95D1F7C701BE01A0
:103CD0000E94652A6F01E12CF12CA7019601260FA5
:103CE000371F411D511DC501B4010E948D2A690174
:103CF0007A01E0918600F0918700CA01B9010E9423
:103D0000472A9B01AC01DF010E94D32A9B01AC0131
:103D1000C701B6010E94472ADC01CB012FE0B6950E
:103D2000A795979587952A95D1F7009186001091D0
:103D3000870020E030E0081719072A073B0728F41E
:103D40006091860070918700CB01BC0170938B005D
:103D500060938A00DF91CF911F910F91FF90EF90B8
:103D6000DF90CF90BF90AF909F908F90089508956F
:103D70000E94FD1D82E28093800089E18093810092
:103D80008FEF9FEF90938700809386000C94F11C37
:103D90006E9A2EB12F7B3EB130644FB7F894FC0180
:103DA000CB01880F991F680F791F6E0F7F1FE617D1
:103DB000F70789F0819198E03EB9000000C087FFC5
:103DC0002EB9880F000000C000C000C02EB900C08E
:103DD0009A9591F7ECCF4FBF8FE594E00197F1F7FB
:103DE00000C000000895CF93DF93EC01FB018281B6
:103DF000882309F43CC1C430FDE5DF0760F4CB3F04
:103E00009CE5D90788F49E0122503C4524313105B8
:103E100008F02EC109C0C236EDE5DE0729F0C63A2A
:103E2000FDE5DF0709F024C10E94160E9093F3020E
:103E30008093F202C1318CE5D80709F4C6C008F0BE
:103E400042C0C930ECE5DE0709F49BC000F5C5307F
:103E50008CE5D80709F485C078F4C330ECE5DE07BB
:103E600009F478C008F07AC0C230DC4509F0F5C02A
:103E70008091F2028160EFC0C7309CE5D90709F458
:103E800078C008F07AC08091F2028061E4C0CD3041
:103E9000FCE5DF0709F487C058F4CB309CE5D9076F
:103EA00009F479C008F07BC08091F20288606FC08D
:103EB000CF30FCE5DF0709F480C008F082C08091B4
:103EC000F202877FC8C0CE3F9CE5D90709F471C0D4
:103ED00000F5C531FCE5DF0709F485C068F4C3319E
:103EE0009CE5D90709F475C008F095C00E94C70782
:103EF0008091F2028F77AFC0CC3FFCE5DF07A9F1DC
:103F000008F054C0CB3FDC4509F0A7C08091F30214
:103F100040C0C230EDE5DE0709F489C058F4C11590
:103F20008DE5D80709F45AC008F069C08091F30202
:103F300082602FC0C236EDE5DE0709F47CC0C63AC8
:103F4000FDE5DF0709F481C0C330DD4509F085C018
:103F500080E06EC08091F20282607DC08091F202AA
:103F600016C08091F202886076C08091F302826070
:103F70004FC08091F20280626EC08091F202806434
:103F80006AC00E94C7078091F202806864C08460A2
:103F900062C081603DC08091F2028E7F5CC08091E2
:103FA000F2028D7F58C08091F20216C08091F30218
:103FB00018C08091F3028D7F2BC08091F2028F7E1A
:103FC0004AC08091F2028F7D46C08091F2028F7BC1
:103FD00042C08091F202877F8B7F3DC08091F302C7
:103FE0008D7F8E7F15C08091F20282FB222720F9FF
:103FF00091E0922790FB82F990FB83F92CC080918D
:10400000F302982F909591708E7F892B90FB81F908
:104010008093F30222C00E94C7078091F20287FBBF
:10402000222720F991E0922790FB87F914C081E0C4
:104030000E94AD0E12C08091F20284FB222720F96B
:1040400091E0922790FB84F906C08091F202982FAC
:10405000909590FB80F98093F2028091F20290910A
:10406000F3020E94270E0E94C70780E001C081E092
:10407000DF91CF910895CF93DF9386319C4541F531
:10408000EB010E941A0D982F8A8120910201309134
:104090000301882379F09A7A81E009F480E0809323
:1040A000C102911102C069E201C065E3C9010E9429
:1040B00031220AC08091C102811102C069E201C0AF
:1040C00065E3C9010E943C220E945C0D80E001C0B2
:1040D00081E0DF91CF9108950F931F93CF93DF93EA
:1040E000C42FD22FFC0182818823C9F04093C402DF
:1040F0000E94F5229093C3028093C20280E28C0F4B
:10410000883008F057C0C77081E001C0880FCA9599
:10411000EAF7DF91CF911F910F910C9424058091C4
:10412000C402481330C08091C2029091C3020E9421
:104130000D23883C910538F510E21D0FCD17B9F01D
:1041400080E28C0F883040F4C77081E001C0880F96
:10415000CA95EAF70E942B05183028F581E09D2FBB
:10416000977001C0880F9A95EAF70E942405802F66
:104170000E941B051830F0F4D77081E001C0880F51
:10418000DA95EAF70AC080E28C0F883098F4C7709D
:1041900081E001C0880FCA95EAF7DF91CF911F91A6
:1041A0000F910C942B05802FDF91CF911F910F91D0
:1041B0000C941B05DF91CF911F910F9108950F93E0
:1041C0009C01CB01243F4CE5340731F188F4293DB3
:1041D000FCE53F07D9F02A3D4CE5340779F1283D4D
:1041E0003C45A9F506E221EE41EE68ED7CE52BC0E9
:1041F000263FFCE53F07E1F0A8F0273F3C4539F5B5
:1042000007E225EE46EE67EF7CE51DC007E225EEEE
:1042100045EE69ED7CE517C006E221EE40EE64EF65
:104220007CE511C007E225EE44EE65EF7CE50BC0AE
:1042300006E221EE42EE66EF7CE505C008E221E0F1
:1042400045EE6AED7CE50E946C2080E008C0FC0130
:104250008281882319F01092C40201C081E00F917D
:1042600008959093C7018093C60108959093CA0260
:104270008093C9020895E091C902F091CA02309773
:1042800021F00190F081E02D099480E00895E09103
:10429000C902F091CA02309799F020912B01222394
:1042A00059F02091F20227FF07C0DC012C911196F2
:1042B0002C93119726E02C930280F381E02D099432
:1042C0000895E091C902F091CA02309739F022E0D6
:1042D000DC012C930480F581E02D09940895209150
:1042E000C7023091C8022817390771F09093C802AD
:1042F0008093C702E091C902F091CA02309721F081
:104300000680F781E02D099408952091C50230912F
:10431000C6022817390771F09093C6028093C50230
:10432000E091C902F091CA02309721F00084F18532
:10433000E02D09940895FC01329680912B01882389
:1043400031F08091F20287FF02C09EE101C096E049
:1043500080E0915028F021912223D9F38F5FF9CF8B
:104360000895662351F120912B012223E9F0209139
:10437000F20227FF19C0462F4695469546954E31C5
:10438000E0F4677021E030E002C0220F331F6A952D
:10439000E2F7FC01E40FF11D828190E0282339232C
:1043A00081E0232B69F409C0FC0132960896219123
:1043B000621729F0E817F907D1F780E0089581E046
:1043C00008959C01FC0132969FEF80E041914617D1
:1043D00089F09F3F19F4411101C0982F8F5F8630FB
:1043E000A9F79F3F39F0F901E90FF11D97FDFA9503
:1043F0006283089508959C012A5F3F4FFC0142812A
:10440000461301C01282019682179307B9F70895E7
:10441000262F2695269526952E3168F4FC01E20F6D
:10442000F11D677021E030E001C0220F6A95EAF7C4
:104430008281282B22830895262F2695269526955E
:104440002E3170F4FC01E20FF11D677021E030E0C5
:1044500001C0220F6A95EAF72095828128232283E2
:10446000089520912B01222329F02091F20227FDAB
:104470000C9408220C94E12120912B01222329F095
:104480002091F20227FD0C941C220C94FB21209118
:104490002B01FC013296222331F08091F20287FF3A
:1044A00002C08EE101C086E0DF011D928A95E9F726
:1044B000089508950C94592283E08093CB020C94C4
:1044C0005A22811102C081E001C082E08093CB02B8
:1044D0000C945A220C94612281E08093CB020C94BC
:1044E0005A220C946C2208950C9473220C9474221A
:1044F0000C9473220C9473220C947322CF930E9419
:104500007A220E94B7120E947822C0E08C2F0E946B
:10451000E111892B29F4CF5FC930C1F780E001C0D8
:1045200081E0CF91089508951F920F920FB60F92D8
:1045300011248F939F93AF93BF938091CC028111ED
:1045400013C08091600390916103A0916203B091C8
:1045500063034196A11DB11D809360039093610395
:10456000A0936203B0936303BF91AF919F918F912A
:104570000F900FBE0F901F901895809168038430A4
:1045800031F10E94E5031092CC0220E488E190E032
:104590000FB6F894A895809360000FBE209360003A
:1045A00083B7817F846083BF83B7816083BF789442
:1045B000889583B78E7F83BF0FB6F894A8958091B6
:1045C0006000886180936000109260000FBE0895C3
:1045D0000E94C7070C94EC0382E084BD93E095BD74
:1045E0009AEF97BD80936E0008952FB7F89480914D
:1045F000600390916103A0916203B09163032FBFA8
:1046000008952FB7F89460916003709161038091D1
:104610006203909163032FBF08959C014FB7F894F4
:104620008091600390916103A0916203B091630354
:104630004FBF821B930B089578941F920F920FB671
:104640000F9211248F939F93AF93BF938091600338
:1046500090916103A0916203B09163030196A11D43
:10466000B11D8093600390936103A0936203B093A4
:104670006303BF91AF919F918F910F900FBE0F90E9
:104680001F90189581E08093E00080E28093D8002D
:104690001092C9008FE19EE40197F1F700C000007D
:1046A00087E090EBDC018093710390937203A093F9
:1046B0007303B09374039CE088E10FB6F894A89557
:1046C000809360000FBE90936000FFCF8091F00256
:1046D0000895089522E02093E9002FEF3091E8003B
:1046E000215035FD06C035ED3A95F1F70000211156
:1046F000F5CF2091E80025FF0BC040E050E066E0D8
:1047000070E00E94A9258091E8008E778093E800F0
:104710000895CF93DF9320912B01222339F020912C
:10472000F20227FF03C060E222E002C068E021E05D
:104730002093E9002FEF3091E800215035FD06C0AD
:1047400035ED3A95F1F700002111F5CF2091E80001
:1047500025FF1DC0EC0180912B01811105C040E0B7
:1047600050E068E070E003C070E040E050E0CE014F
:104770000E94A9258091E8008E778093E80080E26E
:10478000FE01A0EDB2E001900D928A95E1F7DF9174
:10479000CF9108958093CD027093CF026093CE02A3
:1047A00080916803843001F582E08093E9008FEF07
:1047B0009091E800815095FD06C095ED9A95F1F72E
:1047C00000008111F5CF8091E80085FF0DC040E029
:1047D00050E063E070E08DEC92E00E94A9258091AA
:1047E000E8008E778093E8000895BC0184E00C9483
:1047F000CA23BC0183E00C94CA2380916703811112
:1048000009C00E943A270E9497278091E2008460A5
:104810008093E20008951092670308950C9471222A
:104820006091640381E0611101C080E00C945C221E
:104830009091680381E0943009F080E06091640316
:104840000C94612242E061EC81E00E94B32642E2D6
:1048500061EC82E00E94B3269091680381E094307D
:1048600009F080E0609164030C946A2280916A03ED
:10487000833009F461C030F4813071F0823009F482
:104880009AC008958A3009F486C08B3009F46CC050
:10489000893009F0A8C020C080916903813A09F0ED
:1048A000A2C08091E800877F8093E80080916D032B
:1048B00090916E03892B21F460E280ED92E003C0B9
:1048C00060E080E090E070E00E94F4258091E800D4
:1048D0008B778093E800089580916903813209F015
:1048E00082C080916D0390916E03029708F07BC0A7
:1048F0008091E800877F8093E8008091E80082FD46
:1049000005C0809168038111F8CF6DC02091F3003C
:104910008091F20090E0922B029731F48091F100A7
:10492000813011F0863021F48091F1008093F00203
:104930008091E8008B7753C080916903813A09F038
:1049400052C080916D0390916E03892B09F04BC08A
:104950008091E800877F8093E8008091E80080FFE5
:10496000FCCF80912B0136C0809169038132D9F54B
:1049700080916D0390916E03892BA9F58091E800D9
:10498000877F8093E8000E94E82680916B038093E4
:104990002B010C94C70780916903813221F5809126
:1049A000E800877F8093E8000E94E82680916C03EE
:1049B0008093F102089580916903813AA1F4809176
:1049C000E800877F8093E8008091E80080FFFCCFBB
:1049D0008091F1028093F1008091E8008E778093BE
:1049E000E8000C94E826089584B7877F84BF0FB64B
:1049F000F894A8958091600088618093600010927F
:104A000060000FBE90E080E80FB6F89480936100DC
:104A1000909361000FBE0C946C220E943A270E9472
:104A20009727E2EEF0E080818460808378940C9494
:104A30002C2A8FE191E00C94362180916803853017
:104A4000A9F480916803853079F40E94BD22809199
:104A500066038823B1F30E947E22882391F30E948B
:104A600093250E94C707EDCF0C94E822089508957E
:104A70000C943A25292F332723303105C9F060F4EF
:104A80002130310581F02230310509F044C08BE33B
:104A900090E027E834E043C021323105E1F02232D2
:104AA000310549F138C082E190E022EC34E037C0B2
:104AB00099278130910549F028F0029761F5E7E5E3
:104AC000F4E005C0E3E8F4E002C0E3E6F4E084913A
:104AD00090E09F0124C06115710541F061307105BE
:104AE000D1F489E090E022EB34E019C089E090E055
:104AF00029E934E014C06115710541F06130710598
:104B000051F486EB90E024ED34E009C080E490E0BD
:104B10002AE835E004C080E090E020E030E0FA01CF
:104B200031832083089580E189BD82E189BD09B484
:104B300000FEFDCF8091D8008F7D8093D8008091BA
:104B4000E00082608093E0008091E00081FDFCCF76
:104B50000895CF92DF92EF92FF920F931F93CF931E
:104B6000DF93EC018B017A010E940727811133C08A
:104B7000E114F10439F0F70180819181081B190BD0
:104B8000C80FD91FC12CD12C0115110519F1809125
:104B9000E80085FD16C08091E8008E778093E800DC
:104BA000E114F10449F0F70180819181C80ED91E0A
:104BB000D182C08285E00FC00E940727882321F39D
:104BC0000AC089918093F10001501109FFEFCF1ABB
:104BD000DF0ADACF80E0DF91CF911F910F91FF9034
:104BE000EF90DF90CF90089520916F033091700384
:104BF0002617370748F06115710539F42091E80050
:104C00002E772093E80001C0B901FC0120E0611576
:104C1000710579F1809168038823F1F18530F1F114
:104C20008091E80083FD3CC08091E80082FD2EC0A9
:104C30008091E80080FFEBCF2091F3008091F2009B
:104C400090E0922B6115710551F08830910538F490
:104C500021912093F100615071090196F3CF21E079
:104C6000089709F020E08091E8008E778093E800B3
:104C7000CECF2111CFCF0AC080916803882361F085
:104C8000853061F08091E80083FD0AC08091E800E2
:104C900082FFF2CF80E0089582E0089583E00895D6
:104CA00081E0089520916F03309170032617370734
:104CB00048F06115710539F42091E8002E772093B2
:104CC000E80001C0B901FC0120E06115710591F116
:104CD00080916803882309F440C0853009F43FC0FF
:104CE0008091E80083FD3DC08091E80082FD2FC0E7
:104CF0008091E80080FFE9CF2091F3008091F200DD
:104D000090E0922B6115710559F08830910540F4BF
:104D100024912093F1003196615071090196F2CFF0
:104D200021E0089709F020E08091E8008E778093D9
:104D3000E800CBCF2111CCCF0AC080916803882333
:104D400061F0853061F08091E80083FD0AC08091B8
:104D5000E80082FFF2CF80E0089582E0089583E0CA
:104D6000089581E00895982F973068F59093E900B1
:104D7000981739F07091EC002091ED005091F000FF
:104D800003C0242F762F50E021FD02C09F5FECCF9F
:104D90003091EB003E7F3093EB003091ED003D7F92
:104DA0003093ED003091EB0031603093EB00709365
:104DB000EC002093ED005093F0002091EE0027FDD1
:104DC000E5CF80E008958F708093E90081E0089539
:104DD0008091690387FF11C08091E80082FD05C0C2
:104DE000809168038111F8CF11C08091E8008B7722
:104DF0000BC080916803882349F08091E80080FF10
:104E0000F8CF8091E8008E778093E8000895209194
:104E1000E4003091E50095E64091EC00842F81702C
:104E200040FF23C08091E80080FD1DC08091680391
:104E3000882399F0853099F08091EB0085FD11C0B1
:104E40004091E4005091E5002417350729F3915073
:104E500011F09A01E1CF84E0089582E0089583E0A3
:104E6000089581E0089580E008954091E80042FFB0
:104E7000DDCF08950E94A8270E94B027E0EEF0E061
:104E8000808181608083E8EDF0E080818F7780838E
:104E900019BCA7EDB0E08C918E7F8C9380818F7EC2
:104EA00080831092670308950F931F93CF93DF932E
:104EB0000E94A8270E94B027C8EDD0E088818F7794
:104EC000888388818068888388818F7D888319BCE6
:104ED00010926803109264031092660310926503A7
:104EE00000EE10E0F80180818B7F808388818160F3
:104EF000888342E060E080E00E94B326E1EEF0E0CB
:104F000080818E7F8083E2EEF0E08081816080830B
:104F1000808188608083F80180818E7F8083888192
:104F200080618883DF91CF911F910F910895E8ED03
:104F3000F0E080818F7E8083E7EDF0E0808181600A
:104F4000808384E082BF81E0809367030C945427C0
:104F5000E8EDF0E080818E7F80831092E20008957A
:104F60001092DA001092E10008951F920F920FB68E
:104F70000F9211242F933F934F935F936F937F93DF
:104F80008F939F93AF93BF93EF93FF938091E10033
:104F900082FF0BC08091E20082FF07C08091E10098
:104FA0008B7F8093E1000E942B2A8091DA0080FFA2
:104FB0001FC08091D80080FF1BC08091DA008E7FD7
:104FC0008093DA008091D90080FF0DC080E189BD17
:104FD00082E189BD09B400FEFDCF81E080936803C2
:104FE0000E94FD2305C019BC109268030E940B2487
:104FF0008091E10080FF19C08091E20080FF15C020
:105000008091E2008E7F8093E2008091E2008061D7
:105010008093E2008091D80080628093D80019BC10
:1050200085E0809368030E9410248091E10084FF52
:1050300030C08091E20084FF2CC080E189BD82E114
:1050400089BD09B400FEFDCF8091D8008F7D80938B
:10505000D8008091E1008F7E8093E1008091E20092
:105060008F7E8093E2008091E20081608093E20075
:1050700080916403882311F084E007C08091E300ED
:1050800087FD02C081E001C083E0809368030E9435
:1050900018248091E10083FF29C08091E20083FF02
:1050A00025C08091E100877F8093E10082E08093BA
:1050B0006803109264038091E1008E7F8093E10089
:1050C0008091E2008E7F8093E2008091E200806117
:1050D0008093E20042E060E080E00E94B32680918D
:1050E000F00088608093F0000E940E24FF91EF9101
:1050F000BF91AF919F918F917F916F915F914F91F0
:105100003F912F910F900FBE0F901F9018951F92F7
:105110000F920FB60F9211242F933F934F935F93EB
:105120006F937F938F939F93AF93BF93CF93DF93AF
:10513000EF93FF93C091E900CF708091EC00D82FDE
:10514000D17080FDD0E81092E9008091F000877F57
:105150008093F00078940E94CB281092E90080910F
:10516000F00088608093F000CD2BCF70C093E900F1
:10517000FF91EF91DF91CF91BF91AF919F918F916F
:105180007F916F915F914F913F912F910F900FBE43
:105190000F901F9018951F93CF93DF93CDB7DEB775
:1051A000AA970FB6F894DEBF0FBECDBFE9E6F3E0D5
:1051B0008091F100819323E0E137F207C9F70E9463
:1051C00036248091E80083FF2EC18091690390917D
:1051D0006A03492F50E04A30510508F024C1FA0112
:1051E000EE59FF4F0C94AF2A803821F0823809F035
:1051F0001AC108C08091650390916603992389F0D4
:1052000082600FC080916D038F70873008F00BC1F2
:105210008093E9008091EB0085FB882780F910924C
:10522000E9009091E800977F9093E8008093F10067
:105230001092F100D1C0282F2D7F09F0F4C08823EF
:1052400019F0823061F0EFC080916B03813009F07A
:10525000EAC0933009F080E0809366032EC080910D
:105260006B0381112AC080916D038F702FEF280F7F
:10527000263008F0D8C08093E9002091EB0020FF91
:105280001CC0933021F48091EB00806214C0909197
:10529000EB0090619093EB0021E030E0A90102C0A7
:1052A000440F551F8A95E2F74093EA001092EA00F6
:1052B0008091EB0088608093EB001092E900809170
:1052C000E800877F8093E8000E94E826ACC0811147
:1052D000AAC010916B031F778091E3008078812B27
:1052E0008093E3008091E800877F8093E8000E942C
:1052F000E8268091E80080FFFCCF8091E300806881
:105300008093E300111102C082E001C083E080932A
:10531000680389C08058823008F085C080916B0393
:1053200090916C038C3D53E0950779F583E08A8377
:105330008AE289834FB7F894DE01139620E03EE0BD
:1053400051E2E32FF0E050935700E49120FF03C0B7
:10535000E295EF703F5FEF708E2F90E0EA3010F033
:10536000C79601C0C0968D939D932F5F243149F756
:105370004FBF8091E800877F8093E8006AE270E089
:10538000CE0101960E94F42516C060916D037091C4
:105390006E03AE014F5F5F4F0E943825BC01892B21
:1053A00009F441C09091E800977F9093E8008981CB
:1053B0009A810E9452268091E8008B778093E800C2
:1053C00032C0803881F58091E800877F8093E800C3
:1053D000809164038093F1008091E8008E7772CF12
:1053E000811121C080916B0390916C0399270297E2
:1053F000D4F48091E800877F8093E80080916B036C
:10540000809364030E94E82680916403811106C0A2
:105410008091E30087FD02C081E001C084E08093B9
:1054200068030E9422248091E80083FF0AC08091D3
:10543000E800877F8093E8008091EB008062809392
:10544000EB00AA960FB6F894DEBF0FBECDBFDF917A
:10545000CF911F9108950895CF9380916803882379
:10546000A1F0C091E900CF709091EC00892F81707C
:1054700090FD80E8C82B1092E9008091E80083FD40
:105480000E94CB28CF70C093E900CF910895DB0133
:105490008F939F930E94D32ABF91AF91A29F800DBB
:1054A000911DA39F900DB29F900D1124089587FB2D
:1054B000082E062687FD819567FD61950E94E62AE4
:1054C0000EF4919507FC81950895AA1BBB1B51E131
:1054D00007C0AA1FBB1FA617B70710F0A61BB70B64
:1054E000881F991F5A95A9F780959095BC01CD0109
:1054F000089597FB072E16F4009407D077FD09D086
:105500000E94652A07FC05D03EF4909581959F4F37
:105510000895709561957F4F0895A1E21A2EAA1BF8
:10552000BB1BFD010DC0AA1FBB1FEE1FFF1FA21753
:10553000B307E407F50720F0A21BB30BE40BF50B50
:10554000661F771F881F991F1A9469F760957095D9
:10555000809590959B01AC01BD01CF010895EE0FA0
:10556000FF1F0590F491E02D09940E94BD2A33237A
:1055700012F48A1B9B0B0C94CE2AA29FB001B39FFE
:10558000C001A39F700D811D1124911DB29F700D4C
:10559000811D1124911D08950E94BD2AB7FF089511
:1055A000821B930B08950E94BD2AA59F900DB49F66
:1055B000900DA49F800D911D11240895B7FF0C94A8
:1055C000D32A0E94D32A821B930B0895991B79E05A
:1055D00004C0991F961708F0961B881F7A95C9F783
:1055E00080950895FC014150504030F0019006161E
:1055F000D1F73197CF010895882799270895FB01A6
:10560000DC0104C08D910190801921F4415050407B
:10561000C8F7881B990B0895F999FECF92BD81BDFB
:10562000F89A992780B50895A6E1B0E044E050E0EB
:105630000C94462BA8E1B0E042E050E00C94462BDD
:10564000262FF999FECF92BD81BDF89A019700B43B
:10565000021639F01FBA20BD0FB6F894FA9AF99ADB
:105660000FBE08950396272F0E94212B0E94202B06
:10567000252F0E94212B242F0C94212B0196272FBC
:105680000E94212B0C94202BDC01CB01FC01F99909
:10569000FECF06C0F2BDE1BDF89A319600B40D927E
:0C56A00041505040B8F70895F894FFCF37
:1056AC00C8006802280850011E0A140101010200FA
:1056BC001600161601191A1B1C1D1E1F202122660E
:1056CC002389236A23F923F523692301E200E900E6
:1056DC00EA00B500B600B700CD008301CC008A010A
:1056EC0092019401210223022402250226022702A0
:1056FC002A02B300B4006F007000818283E200E9DB
:10570C0000EA00B500B600B700CD008301CC008ADA
:10571C000192019401210223022402250226022770
:10572C00022A02B300B4006F00700081828395944A
:10573C0096973435F56667F730313233379091925E
:10574C009300010202020206060609090909090969
:10575C000F0F0F0F0F0F15151518191919191919F6
:06576C001919191923248C
:00000001FF
